:020000021000EC
:10F800000C944AFC0C9469FC0C9469FC0C9469FC03
:10F810000C9469FC0C9469FC0C9469FC0C9469FCD4
:10F820000C9469FC0C9469FC0C9469FC0C9469FCC4
:10F830000C9469FC0C9469FC0C9469FC0C9469FCB4
:10F840000C9469FC0C9469FC0C9469FC0C9469FCA4
:10F850000C9469FC0C9469FC0C9469FC0C9469FC94
:10F860000C9469FC0C9469FC0C9469FC0C9469FC84
:10F870000C9469FC0C9469FC0C9469FC0C9469FC74
:10F880000C9469FC0C9469FC0C9469FC0C9469FC64
:10F890000C9469FC11241FBECFEFD0E1DEBFCDBFB9
:10F8A00011E0A0E0B1E0E8E7FFEF01E00BBF02C02C
:10F8B00007900D92A030B107D9F711E0A0E0B1E0B8
:10F8C00001C01D92A130B107E1F70E9487FD0C94A1
:10F8D000BAFF0C9400FC0F931F93CF93DF938C011E
:10F8E000EA016534C9F488819981AA81BB8181BD0F
:10F8F000292F3A2F4B2F552722BD0196A11DB11D4F
:10F9000088839983AA83BB83F89A80B50E9478FF85
:10F910000150104041F73AC0663409F037C0888181
:10F920009981AA81BB81880F991FAA1FBB1F888359
:10F930009983AA83BB8388819981AA81BB81ABBF4C
:10F94000FC0187910E9478FF88819981AA81BB81FF
:10F950000196A11DB11DABBFFC0187910E9478FFEC
:10F9600088819981AA81BB810296A11DB11D8883DE
:10F970009983AA83BB8302501040E9F6B695A795F8
:10F980009795879588839983AA83BB83DF91CF91CD
:10F990001F910F9108955F926F927F928F929F9225
:10F9A000AF92BF92CF92DF92EF92FF920F931F938D
:10F9B000DF93CF93CDB7DEB7C050D1400FB6F894E8
:10F9C000DEBF0FBECDBF3C014A016534B9F57E01F3
:10F9D0000894E11CF11C67015701A80EB91E05C06F
:10F9E0000E9484FFF60181936F01CA14DB04C1F702
:10F9F00007B600FCFDCF1EC0F40120813181428199
:10FA0000538121BDBB27A52F942F832F82BDF701E2
:10FA1000808180BDFA9AF99AF999FECF2F5F3F4F06
:10FA20004F4F5F4FF4012083318342835383089407
:10FA3000E11CF11CEC14FD04F9F651C0663411F020
:10FA40008FE34EC0FA01A080B180C280D380AA0C9F
:10FA5000BB1CCC1CDD1CA082B182C282D382552487
:10FA600053940E9484FF082F10E00E9484FFF40149
:10FA70002081318142815381F82EEE240E291F29E5
:10FA80000801F90140935B0050925700E89511245A
:10FA90002E5F3F4F4F4F5F4FF401208331834283EE
:10FAA00053838EEF9FEF680E791E61147104C9F6BF
:10FAB00085E0F501C0925B0080935700E89507B69A
:10FAC00000FCFDCF81E180935700E895569547955E
:10FAD00037952795F40120833183428353838DE04A
:10FAE000C050DF4F0FB6F894DEBF0FBECDBFCF9131
:10FAF000DF911F910F91FF90EF90DF90CF90BF901B
:10FB0000AF909F908F907F906F905F9008952F920D
:10FB10003F924F925F926F927F928F929F92AF929D
:10FB2000BF92CF92DF92EF92FF920F931F93DF93DA
:10FB3000CF9300D000D0CDB7DEB70E94A1FFA19A2D
:10FB40000E9471FF9199ACC10E9495FF09E02224A7
:10FB500033242E010894411C511C0E9484FF182F4D
:10FB60000E9495FF113611F489E597C1113479F49B
:10FB70000E9484FF182F0E9484FFD12ECC2490E095
:10FB80008C299D29AA2797FDA095BA2FD8C0153694
:10FB9000E1F480E090E0A0E0B0E00EC007B600FC29
:10FBA000FDCF23E0FC01A0935B0020935700E89574
:10FBB00080509F4FAF4FBF4F803068EF960761E096
:10FBC000A60760E0B60750F3BAC0123629F489E5FB
:10FBD0000E9478FF81E028C1123499F40E9484FFCA
:10FBE000182F0E9484FFB12EAA24E82EFF24EA28B1
:10FBF000FB280E9484FF682FC701A2010E94CBFC52
:10FC00004CC1173699F40E9484FF182F0E9484FF7C
:10FC1000912E8824E82EFF24E828F9280E9484FFEA
:10FC2000682FC701A2010E946BFC97CF123519F50E
:10FC300007B600FCFDCF81E180935700E8958981EC
:10FC40009A81AB81BC81880F991FAA1FBB1F0196A7
:10FC5000A11DB11DABBFFC0187910E9478FF898176
:10FC60009A81AB81BC81880F991FAA1FBB1FABBFB4
:10FC7000FC01879177C0133629F40E9484FFE82E97
:10FC8000FF24DEC01334E9F40E9484FF782E66243A
:10FC9000E628F72807B600FCFDCF89819A81AB8161
:10FCA000BC819C01AD01220F331F441F551F61E031
:10FCB0000701F90140935B0060935700E895112418
:10FCC0003BC01D36F9F489819A81AB81BC818030BB
:10FCD0002CEF920720E0A20720E0B20720F08FE38C
:10FCE0000E9478FFADC007B600FCFDCF880F991FBA
:10FCF000AA1FBB1F65E0FC01A0935B006093570047
:10FD0000E8959EC0143401F507B600FCFDCF89814B
:10FD10009A81AB81BC8181BD892F9A2FAB2FBB27E4
:10FD200082BD0E9484FF80BDFA9AF99AF999FECFAC
:10FD300089819A81AB81BC810196A11DB11D898306
:10FD40009A83AB83BC837CC01436D1F489819A81B9
:10FD5000AB81BC8181BD892F9A2FAB2FBB2782BD80
:10FD6000F89A80B50E9478FF89819A81AB81BC8125
:10FD70000196A11DB11D89839A83AB83BC83EDCE0F
:10FD80001C3661F407B600FCFDCF0E9484FFE1E061
:10FD9000F0E0082E00935700E89552C0123749F45E
:10FDA00007B600FCFDCFE1E0F0E00093570084913E
:10FDB00074C0163449F407B600FCFDCFE0E0F0E073
:10FDC00000935700849169C01E3449F407B600FCC3
:10FDD000FDCFE3E0F0E00093570084915EC0113561
:10FDE00049F407B600FCFDCFE2E0F0E000935700D5
:10FDF000849153C0103521F11C3411F1153469F48C
:10FE000007B600FCFDCF81E180935700E8958DE0B7
:10FE10000E9478FFF1010995A0CE103711F483E517
:10FE20003CC0143729F484E40E9478FF80E035C098
:10FE3000183721F0193711F0143521F40E9484FF8E
:10FE40008DE02BC01335A1F481E40E9478FF86E594
:10FE50000E9478FF82E50E9478FF82E40E9478FF8A
:10FE60008FE40E9478FF8FE40E9478FF84E515C03C
:10FE7000163529F481E30E9478FF85E30EC013371D
:10FE800041F481E80E9478FF87E90E9478FF8EE1C3
:10FE900004C01B3109F461CE8FE30E9478FF5DCE70
:10FEA00007B600FCFDCF81E180935700E895E0E0C4
:10FEB000F0E009950F900F900F900F90CF91DF9188
:10FEC0001F910F91FF90EF90DF90CF90BF90AF9078
:10FED0009F908F907F906F905F904F903F902F906A
:10FEE000089580E28093CC0088E18093C900089552
:10FEF0008093CE008091C80086FFFCCF8091C8001F
:10FF000080648093C80008958091C80087FFFCCF6B
:10FF10008091CE00089510926E0010926F001092A2
:10FF2000700010927100789408958091000191E022
:10FF3000892780930001882311F05E9A08955E98C6
:10FF400008959FEF92B911B82FE025B987EF84B9D2
:10FF500018B897B98DE38BB98AEC8AB986E88EB95F
:10FF60008BEF8DB921BB80EF80BB8EE184BB89E133
:08FF700083BB0895F894FFCF54
:040000031000F800F1
:00000001FF
